S02B0000443A2F7573722F6665617365722F736F6674776172652F4F70656E424C542F5461726765742F44657D
S1130000680600207B010000B50E0000B50E00005C
S1130010B50E0000B50E0000B50E0000B50E0000D0
S1130020B50E0000B50E0000B50E0000B50E0000C0
S1130030B50E0000B50E0000B50E0000B50E0000B0
S1130040B50E0000B50E0000B50E0000B50E0000A0
S1130050B50E0000B50E0000B50E0000B50E000090
S1130060B50E0000B50E0000B50E0000B50E000080
S1130070B50E0000B50E0000B50E0000B50E000070
S1130080B50E0000B50E0000B50E0000B50E000060
S1130090B50E0000B50E0000B50E0000B50E000050
S11300A0B50E0000B50E0000B50E0000B50E000040
S11300B0B50E0000B50E0000B50E0000B50E000030
S11300C0B50E0000B50E0000B50E0000B50E000020
S11300D0B50E0000B50E0000B50E0000B50E000010
S11300E0B50E0000B50E0000B50E0000B50E000000
S11300F072B64B484B4901604B498D464B484C49BD
S11301004C4A00F07BF84C484C494D4A00F076F8D4
S11301104C484D494D4A00F071F84D484D494E4AFE
S113012000F06CF84D484E494E4A00F067F84E48CE
S11301304E494F4A00F062F84E484F49002200F001
S113014068F84E484E49091A082903DB0022026068
S1130150043001603F484049884205D002680430B9
S113016003B4904703BCF7E700208646EC4601F051
S1130170BDF900200021434A904772B62A498D46B2
S11301802A482B492B4A00F039F82B482B492C4A92
S113019000F034F82B482C492C4A00F02FF82C4856
S11301A02C492D4A00F02AF82C482D492D4A00F0FC
S11301B025F82D482D492E4A00F020F82D482E49C7
S11301C0002200F026F82D482D49091A082903DBDE
S11301D000220260043001601E481F49884205D095
S11301E00268043003B4904703BCF7E70020864656
S11301F0EC4600200021234A9047FEE7884207D0BE
S1130200521A05D0037801300B700131013AF9D14B
S11302107047884202D002700130FAE7704700004C
S113022008ED00E00000000068060020701B0000DC
S11302300000002000000020880200008802000066
S113024048170000701B0000000000200000002080
S1130250481700004817000048170000481700001E
S1130260481700004817000048170000481700000E
S11302706D1B000000000020E8040020E8040020BA
S10B028068050020890E00004E
S11302888C4AA0F58013811A013B4A4242EB0102D1
S1130298012B8CBF134642F00103002B40F006816A
S11302A8854BC21A534243EB0203844A904208BF67
S11302B843F00103002B40F0F980814B814AC3EBE2
S11302C8000CDCF1000343EB0C03904208BF43F03D
S11302D80103002B40F0EA807B4B02F57852C11AE7
S11302E84B4243EB0103904208BF43F00103002B48
S11302F840F0DC80754BC21A534243EB0203744A44
S1130308904208BF43F00103002B40F0CF80714BAB
S1130318C3EB000CDCF1000343EB0C030332904203
S113032808BF43F00103002B40F0C0806A4BC11A98
S11303384B4243EB01030C32904208BF43F00103E4
S1130348002B40F0B380654BC3EB000CDCF10003D9
S113035843EB0C033032904208BF43F00103002BF7
S113036840F0A4805E4BC11A4B4243EB0103C032F8
S1130378904208BF43F00103002B40F09780A0F19E
S11303884002534243EB0203B0F1102F08BF43F07D
S11303980103002B40F08A80524B534AC3EB000CF4
S11303A8DCF1000343EB0C03904208BF43F0010364
S11303B8002B7BD14D4B4E4AC11A4B4243EB0103F0
S11303C8904208BF43F00103002B6FD1494BC21A76
S11303D8534243EB0203B0F1101F08BF43F001037B
S11303E8002B63D1444B454AC3EB000CDCF10003FA
S11303F843EB0C03904208BF43F00103002B55D193
S11304083F4BA2F5F072C11A4B4243EB01039042F1
S113041808BF43F00103002B48D13A4B3A4AC3EBD7
S1130428000CDCF1000343EB0C03904208BF43F0DB
S11304380103002B3AD1354BC11A4B4243EB01035C
S11304480332904208BF43F00103002B2ED1304BF6
S1130458C21A534243EB02032E4A904208BF43F0A8
S113046801031BBB2C4BC3EB000CDCF1000343EB77
S11304780C030332904208BF43F00103B3B9A0F15F
S113048820214B42254A43EB0103904208BF43F025
S113049801036BB9A0F10802534243EB0203204A5B
S11304A8904214BF184643F001007047012070477A
S11304B80120704700011000000210000004100021
S11304C80001101000021010000410100050102039
S11304D80100002002000020080000202000002065
S11304E880000020004000100010101000011020AF
S11304F880000030100000300001001000020010DD
S1130508100000102000003001001010020010102C
S11305180800101001000010020000100100102053
S11305280010100010B50446FFF7AAFE20B90948C8
S11305384FF4FC7100F062FF220FA1B2C4F304442B
S113054811FA04F4044B53F822301A6814431C605B
S113055810BD00BFA4170000181800000138FDD111
S1130568704700004A4B70B51A68044612F0E04F11
S113057805D01A68474B1340B3F1805F02D1002CB1
S1130588C0F284804449454A0B68166843F4006302
S113059823F4800546F4006698070D60166001D5BB
S11305A8A10703D5EB0721D5E0071FD464F00303A3
S11305B81D40394B002E1D600DDA06F07003A3F1BF
S11305C830014A4242EB0102702B14BF134642F039
S11305D8010323B906E005F03003302B02D14FF4B0
S11305E8805001E04FF40020FFF7B8FF25F45E5572
S11305F843F2F073234025F070051D43284B294A24
S11306083340294E402126401E4304F0080356EA8D
S1130618C306224B116002F108024BBF1E6015602D
S113062815601E601020FFF799FF204B25F0F86530
S1130638234025F00305620045EA030526F0FC562D
S113064804F0FC5346EA030641BF194B26F480061E
S1130658234045F480054CBF1E4326F080462305FD
S11306680BD4144A4FF400431168480601D4013BE3
S1130678FAD125F4006526F40066074B10201D60A6
S113068810331E60BDE87040FFF768BF70BD00BF3F
S113069800E00F400000FF7060E00F4070E00F4082
S11306A88FDFFF7F58E00F40302000800300C00731
S11306B80000404050E00F40624B70B51A68103398
S11306C81B68002BB4BF03F0700102F0300120292D
S11306D83BD004D871B1102940F0B28010E06029F1
S11306E85FD070295AD0302908BF47F2305040F003
S11306F8A7805CE05449C2F3841051F8200056E006
S11307085249086810F0E04F4ED00C685048204019
S1130718B0F1805F48D00C684D4820404D4CA04251
S113072805D1096889B2022908BF4B483FD0474818
S1130738474904682140494CA14218BF484836D16A
S11307480068474980B2444C23E04049086810F0E7
S1130758E04F2BD00C683E482040B0F1805F25D094
S11307680C683B4820403B4CA04205D1096889B23B
S1130778022908BF3B481AD0344835490468214047
S1130788364CA14218BF384811D100683649354C57
S113079880B200280CBF2046084608E04FF4004009
S11307A805E04FF4800002E0304800E03048002BB8
S11307B802DA13F4006F01E012F4006F28D12D4916
S11307C8224D09682C6814F0E04F43F6E07401EAFE
S11307D804044FEA541405D02E681D4D3540B5F174
S11307E8805F05D1023401F01F056043023504E03F
S11307F8604301F01F0501356D00B0FBF5F011F4FD
S1130808804F18BF4008090448BF800842F480029A
S1130818510216D5002B0DDA590005D51A0503D453
S11308284000C3F3865301E0C3F3C5530133B0FB5F
S1130838F3F070BDC2F3C3520132B0FBF2F070BDE5
S1130848002070BD60E00F404817000000E00F4032
S11308580000FF7000000110001BB7000000031027
S11308680024F400C0C62D0000093D00C0E1E400E6
S11308787038390064E00F40A0F14022534243EB42
S113088802033C4A904208BF43F00103002B6CD199
S1130898394B02F58052C3EB000CDCF1000343EB47
S11308A80C03904208BF43F00103002B5DD1334B86
S11308B802F58052C11A4B4243EB0103904208BF30
S11308C843F00103002B50D12D4B02F58052C3EBAA
S11308D8000CDCF1000343EB0C03904208BF43F027
S11308E80103002B41D1274B02F58052C11A4B4218
S11308F843EB0103904208BF43F00103002B34D1BA
S1130908214B02F58052C3EB000CDCF1000343EBEE
S11309180C03904208BF43F0010333BB1B4B02F5A1
S11309288052C11A4B4243EB0103904208BF43F083
S11309380103D3B9164B02F58052C3EB000CDCF16A
S1130948000343EB0C03904208BF43F0010373B95F
S1130958104B02F58052C11A4B4243EB01039042FB
S113096814BF184643F00100704701207047012066
S1130978704700BF00800540005000400060004000
S113098800700040004002400050024000600240F5
S11309980070024000D0034070B504461646CDB23C
S11309A8FFF76AFF18B91048E42100F027FD022E6A
S11309B803D90D48E62100F021FDD4F8003416F0DF
S11309C8010F14BF2B43AB4304F580621360D4F8C2
S11309D8202416F0020F04F5846314BF154322EA99
S11309E805051D6070BD00BF24180000F0B504465D
S11309F815461F46CEB2FFF73FFF20B94E484FF4C5
S1130A08DD7100F0FBFC6A1E2B1F18BF0123012AAD
S1130A1894BF002303F0010333B10C2D04D04648DE
S1130A284FF4DF7100F0EAFCB7F1080318BF0123A3
S1130A380A2F0CBF002303F00103CBB1B7F10C0359
S1130A4818BF0123092F0CBF002303F001037BB156
S1130A58B7F10B0318BF01230D2F0CBF002303F0BC
S1130A6801032BB127B1344840F2C51100F0C6FC8C
S1130A78D4F8003515F0010F14BF3343B34304F51C
S1130A88A0621360D4F8042515F0020F04F5A063DE
S1130A9814BF3243B24303F104031A60D4F808358F
S1130AA815F0040F14BF3343B34304F5A162136074
S1130AB8D4F8183515F0080F14BF3343B34304F5BD
S1130AC8A3621360D4F80C2517F0010F04F5A06392
S1130AD814BF3243B24303F10C031A60D4F810353F
S1130AE817F0020F14BF3343B34304F5A262136033
S1130AF8D4F8142517F0040F04F5A26314BF324385
S1130B08B24303F104031A60D4F81C2517F0080F44
S1130B1804F5A26303F10C0314BF3243B2431A6011
S1130B28D4F8282504F5A5630FB9164301E022EA91
S1130B3806061E60F0BD00BF2418000030B5044648
S1130B48CDB2FFF799FE20B9084840F21F5100F0D2
S1130B5855FC204629460222FFF71EFF2046294657
S1130B6801220823BDE83040FFF740BF24180000E5
S1130B78830510B5044603D00B48842100F03EFCDD
S1130B880A4B01221A6043F8144C094A143B0833EF
S1130B981A601A689207FCD4064B186810F0010012
S1130BA818BF4FF0FF3010BD9318000014D00F4049
S1130BB8020042A40CD00F402DE9F04105468807F5
S1130BC80C46164603D02848C82100F017FCB10784
S1130BD803D02548C92100F011FC244B01221A60D6
S1130BE8234B1B68DA071ED4224B234F234824497E
S1130BF81A462EE024F07F03CCF8003007E0214B9E
S1130C080434434455F8048B043EC3F8008014F0BC
S1130C187C0801D13B680BB9002EF0D110600B6839
S1130C28DB07FCD405E0184ADFF84CC0174F14481A
S1130C381146002EDED10EE03C6055F804CBC0F816
S1130C4800C01960D2F800C01CF0010FFAD10434B6
S1130C58043E002EF0D10E4B186810F0010018BFA6
S1130C684FF0FF30BDE8F0819318000014D00F4016
S1130C78A0E10F4008D00F4000D00F4004D00F402F
S1130C88010042A400D10F4020D00F4030D00F40C3
S1130C980CD00F40094BC21A534243EB0203084AD3
S1130CA8904208BF43F001032BB9064BC31A5842BC
S1130CB840EB030070470120704700BF00C00040AC
S1130CC800D0004000E0004010B50446FFF7E2FF02
S1130CD820B908484FF4CF7100F090FBE36A43F061
S1130CE81003E362236B43F4407343F0010323636B
S1130CF810BD00BF0619000010B50446FFF7CAFF6F
S1130D0820B909484FF4DF7100F078FBA36918078C
S1130D18FCD4E36A23F01003E362236B23F44073E7
S1130D2823F00103236310BD06190000F0B504463F
S1130D380D4616461F46FFF7ADFF20B92C4840F272
S1130D480D1100F05BFB26B929484FF4877100F0B8
S1130D5855FB284B1A6812F0E04F1DD01968264A33
S1130D680A40B2F1805F17D01968234A0A40234920
S1130D788A4203D11B689BB2022B0DD01D4A1E4B1D
S1130D8811680B401E498B4208D113689BB2002B93
S1130D980CBF1023082302E0102300E00823734348
S1130DA89D4204D2124840F20F1100F027FB20465E
S1130DB8FFF7A2FF236BB5EB061F2BBF23F020031D
S1130DC843F020032363236338BF7608ED00B5FBA3
S1130DD8F6F60136F3096362C6F345060023204696
S1130DE8A662E762A361BDE8F040FFF76DBF00BFEC
S1130DF80619000000E00F400000FF700000011019
S1130E080000031010B50446FFF744FF20B9064854
S1130E1840F2E93100F0F2FAA36913F0200F14BF8D
S1130E280020012010BD00BF0619000010B50446BB
S1130E38FFF730FF20B9064840F2094100F0DEFA16
S1130E48A369DB0654BF20684FF0FF3010BD00BF14
S1130E580619000030B50446CDB2FFF71BFF20B9D0
S1130E68064840F25B4100F0C9FAA369990602D426
S1130E782560012030BD002030BD00BF06190000E8
S1130E8800B50848FFF76EFB0748FFF74BFB4FF028
S1130E9840200321FFF752FE00F0E0FA00F0E9FADF
S1130EA8FCE700BF8003C0010100002001483C2189
S1130EB800F0A4BA7819000000B500F0DFF948B1D1
S1130EC800F006FB044B4FF400521A6042F204038C
S1130ED81B6898475DF804FB08ED00E070B50C4604
S1130EE895B2064607E014F8013B013D06F8013BBC
S1130EF800F001FBADB2002DF5D170BDFFF739B993
S1130F0870B50C4D0646002400F0F5FA2B689E4295
S1130F1809D36A689B189E4205D2064B0C2202FB31
S1130F280434207A70BD01340C35132CECD1FF2025
S1130F3870BD00BF041A00002DE9F14105460068A0
S1130F48FFF7DEFFFF2818D000242F68261DAB59B1
S1130F5804EB0708009300F0CEFA684641460422E1
S1130F68FFF72AFE48B9E259009B9A4206D1B6F522
S1130F78007F3446E9D1012000E00020BDE8F88173
S1130F88114B30B5984204460D4606D0B1F5005FC2
S1130F9805D0FFF7D1FF18B910E00C4C00E01C464F
S1130FA8EB050DD12368AB420BD0204640F8045B17
S1130FB829464FF40072FFF791FF02E0044600E06F
S1130FC80024204630BD00BF000000200402002099
S1130FD82DE9F0431FFA83F8036821F4FE770133FF
S1130FE804460D46164627F0030706D140F8047B4D
S1130FF839464FF40072FFF771FF2368BB4205D0EE
S113100820463946FFF7BCFF044610B3236840F274
S1131018FF19ED1A0435651907F5007700F06BFA26
S1131028231DEB1A4B4506D920463946FFF7A8FF7E
S1131038044680B1051D16F8013B08F1FF381FFA74
S113104888F805F8013BB8F1000FE7D10120BDE8A5
S1131058F083BDE8F083BDE8F0830000034A4FF055
S1131068FF331360024A1360704700BF0402002074
S11310780000002070B504460E461546FFF740FFF1
S1131088FF2815D0601E8019FFF73AFFFF280FD0FC
S113109824F4FE7323F00303B3F5005F0CBF054883
S11310A80548B3B221462A46BDE87040FFF790BF11
S11310B8002070BD00000020040200202DE9F0414A
S11310C80E460446FFF71CFF013C0546A019FFF72E
S11310D817FFA5F1FF030746584240EB0300FF2F13
S11310E808BF40F0010000285DD1BD425CD8002D46
S11310F853D0132F58D82D4E0446B04600F0FBF9B0
S113110898F80830AB4204D10C204443274B1C59AF
S113111806E00134132C08F10C08EFD14FF0FF342A
S1131128DFF88880002500F0E6F998F80830BB421B
S113113805D10C235D431D4B53F8058006E00135AA
S1131148132D08F10C08EED14FF0FF38002500F0FC
S1131158D2F9337ABB4205D1144B0C2202FB053574
S11311686B6804E001350C36132DF0D10023C4EB71
S11311780806F618C6F38F26002509E000F0BBF927
S11311882046FFF7F5FC04F5806448B90135ADB293
S1131198B542F3D30120BDE8F0812846BDE8F081CB
S11311A80020BDE8F0810020BDE8F081041A0000A9
S11311B80F4B01B51A68013217D05A68996842F280
S11311C8F0008918DA6889181A6989185A69891817
S11311D89A698918DA698B185B4201AA42F8043DB6
S11311E804216A46FFF746FF00E0012008BD00BF5E
S11311F80000002042F2040318684FF400531B68EF
S1131208C01842F208031B68C01842F20C031B689A
S1131218C01842F210031B68C01842F214031B687A
S1131228C01842F218031B68C01842F2F0031B6886
S1131238C018D0F1010038BF002070470A4800B533
S11312480368013302D0FFF777FE58B107480368F3
S1131258013306D0FFF770FE003018BF01205DF897
S113126804FB01205DF804FB0000002004020020B8
S1131278FFF7F4BEFFF7FEBEFFF720BFFFF7BABFC4
S113128800B5FFF795FF18B15DF804EBFFF7D6BF7B
S11312985DF804FB054B00224CF24F311A6059608B
S11312A805219A601960024B1A80704710E000E02B
S11312B808040020014B00221A60704710E000E087
S11312C8044B1B68DB0303D5034B1A8801321A80CD
S11312D8704700BF10E000E00804002000B5FFF7E5
S11312E8EFFF024B18885DF804FB00BF08040020D8
S11312F800B50748FFF716F9FFF7DEF90146054878
S11313084FF4614260235DF804EBFFF70FBD00BFA3
S11313180100001000C0004070B5CDB2402D064653
S113132803D91848572100F069F817482946FFF7E8
S113133891FD40B101E000F0DEF81348FFF762FDCB
S11313480028F8D003E00F485A2100F057F8002489
S113135814E000F0D0F8315D0B48FFF77BFD40B195
S113136801E000F0C8F80848FFF74CFD0028F8D061
S113137803E00448622100F041F80134A3B2AB420F
S1131388E7D370BDE81A000000C00040F0B5174C60
S1131398064625785DB91648FFF748FD421C1FD05C
S11313A8144B187001232370134B1D7018E0124D51
S11313B80F482F78FFF73AFD431C13D00D492B78BB
S11313C8CF19787001330A78DBB29A422B700BD1AB
S11313D830460131FFF782FD002323700120F0BD60
S11313E82846F0BD0020F0BD0020F0BD4C040020CC
S11313F800C000400A0400204B040020034B00B541
S11314081860034B196000F076F8FCE750040020DC
S11314185404002010B500F06BF801280FD0084CD4
S11314282378012B0BD1FFF759FF312807D9002363
S11314382370FFF73FFFBDE81040FFF73DBD10BD27
S113144858040020044B012200B51A70FFF722FF4C
S11314585DF804EBFFF7DEBF5804002000B500F088
S113146849F8FFF7EFFFFFF703FF5DF804EB00F01F
S113147809B800B500F03FF800F01AF85DF804EB7D
S1131488FFF7C8BF01B5FF238DF8003000238DF89E
S1131498013000F03BF8FFF72BFF044B1B78012BBE
S11314A802D1684600F050F808BD00BF5904002076
S11314B800B50648FFF76AFF012804D103485DF820
S11314C804EB00F041B85DF804FB00BF5A040020A7
S11314D8704700B5C9B2FFF71FFF5DF804EB00F0D1
S11314E82BB80000014B01221A70704759040020E0
S11314F800F01AB870477047034BFE22DA700222D4
S11315081871A3F8442070479C040020054B00225E
S11315181A709A6483F84320A3F844209A705A7086
S1131528704700BF9C040020024B1878003018BF95
S1131538012070479C040020024B002283F84320BA
S1131548704700BF9C04002070B503780546FF2B44
S1131558784C0FD1E370102301220021237140231A
S113156822706272A27261706171A371E371217257
S113157808227DE02678012E40F0DB80F32B40D052
S113158811D8CF2B00F0B78005D8C92B77D0CC2B36
S113159840F0BA80B6E0D12B00F0A7807CD3D22BE0
S11315A840F0B28093E0FA2B47D006D8F52B0CD044
S11315B811D3F62B40F0A8801FE0FD2B4ED0FE2B54
S11315C859D0FC2B40F0A08046E042783F2A66D8E8
S11315D8201DA16C06E043783F2B60D84168A164C4
S11315E84278201DFFF77AFCFF23E3706A78A36C26
S11315F8D318A3646B78013374E0FF23E370436862
S113160848E0FF23E3700023A06C69681A4603E0EE
S11316181C5C01331219D2B28B42F9D1454B00211B
S1131628DA71120E9A7201221A7108221972597209
S113163859719971A3F8442069E0FF23E3703E4B84
S11316480722A364002323716371A3712372637255
S1131658A372E271082345E0002056E0FF23627874
S1131668E370002362712371A371E371237206226C
S1131678A4F844204BE00023237063703DE0421C2F
S11316883F21A06CFFF7F6FD00283BD0FF23E37051
S1131698A36C3F33A36432E043783E2B01D9222064
S11316A833E0FF23E370A4F84460417821B9FFF7DD
S11316B8E7FD00282BD125E01E4C821CA06CFFF707
S11316C8D9FDF8B16A78A36CD318A3641FE0FF238B
S11316D8E3704022002323716371E3712372637200
S11316E8A2710723A4F8443011E0A06C6968FFF7DD
S11316F8C3FD10B906E0FFF701FCFF23E370A4F86B
S1131708446004E0312000E02020FFF7F5FE094C96
S113171894F84330012B02D11020FFF7EDFEB4F802
S113172844100648012384F84330BDE87040FFF7AD
S1131738D0BE70BD9C040020651B00009F040020DF
S113174840420F0000201C0080841E0000802500F9
S1131758999E36000040380000093D0000803E0094
S113176800004B00404B4C0000204E00808D5B0075
S113177800C05D000080700000127A0000007D0047
S113178880969800001BB7000080BB00C0E8CE001C
S1131798647ADA000024F4000000FA00443A2F7551
S11317A873722F6665617365722F736F66747761E0
S11317B872652F4F70656E424C542F546172676581
S11317C8742F44656D6F2F41524D434D335F4C4D1B
S11317D833535F454B5F4C4D3353383936325F438F
S11317E8726F7373776F726B732F426F6F742F6995
S11317F864652F2E2E2F6C69622F64726976657268
S11318086C69622F73797363746C2E630000000033
S113181800E10F4004E10F4008E10F40443A2F75FE
S113182873722F6665617365722F736F667477615F
S113183872652F4F70656E424C542F546172676500
S1131848742F44656D6F2F41524D434D335F4C4D9A
S113185833535F454B5F4C4D3353383936325F430E
S1131868726F7373776F726B732F426F6F742F6914
S113187864652F2E2E2F6C69622F647269766572E7
S11318886C69622F6770696F2E6300443A2F757311
S1131898722F6665617365722F736F6674776172F0
S11318A8652F4F70656E424C542F5461726765748E
S11318B82F44656D6F2F41524D434D335F4C4D336B
S11318C8535F454B5F4C4D3353383936325F43725F
S11318D86F7373776F726B732F426F6F742F6964B2
S11318E8652F2E2E2F6C69622F6472697665726C6F
S11318F869622F666C6173686C69622E6300443A8E
S11319082F7573722F6665617365722F736F6674B2
S1131918776172652F4F70656E424C542F54617213
S11319286765742F44656D6F2F41524D434D335F86
S11319384C4D33535F454B5F4C4D33533839363236
S11319485F43726F7373776F726B732F426F6F7429
S11319582F6964652F2E2E2F6C69622F6472697645
S113196865726C69622F756172746C69622E6300AA
S1131978443A2F7573722F6665617365722F736F9E
S11319886674776172652F4F70656E424C542F549C
S113199861726765742F44656D6F2F41524D434DD5
S11319A8335F4C4D33535F454B5F4C4D335338399C
S11319B836325F43726F7373776F726B732F426F34
S11319C86F742F6964652F2E2E2F2E2E2F2E2E2FF7
S11319D82E2E2F536F757263652F41524D434D332D
S11319E85F4C4D33532F43726F7373776F726B73FE
S11319F82F766563746F72732E63000000200000F5
S1131A080020000001000000004000000020000049
S1131A180200000000600000002000000300000035
S1131A2800800000002000000400000000A0000066
S1131A38002000000500000000C000000020000095
S1131A480600000000E0000000200000070000007D
S1131A580000010000200000080000000020010030
S1131A6800200000090000000040010000200000E0
S1131A780A00000000600100002000000B000000C4
S1131A8800800100002000000C00000000A00100FC
S1131A98002000000D00000000C00100002000002C
S1131AA80E00000000E00100002000000F0000000C
S1131AB80000020000800000100000000080020006
S1131AC800800000110000000000030000800000F6
S1131AD812000000008003000080000013000000D2
S1131AE8443A2F7573722F6665617365722F736F2D
S1131AF86674776172652F4F70656E424C542F542B
S1131B0861726765742F44656D6F2F41524D434D63
S1131B18335F4C4D33535F454B5F4C4D335338392A
S1131B2836325F43726F7373776F726B732F426FC2
S1131B386F742F6964652F2E2E2F2E2E2F2E2E2F85
S1131B482E2E2F536F757263652F41524D434D33BB
S1131B585F4C4D33532F756172742E63004F70655B
S1081B686E424C540024
S903017B80
